:10800000800CFFFFFFFFFFFFFFFFFF02821EC0A8E3
:10801000750E00750D00750C00750F14E58954F090
:108020004401F589758C4C758A0DD28CD2A9D2AFDA
:108030001281C09080FE1281AF74401281BA90818B
:108040000F1281AF742C1281BAE50E1281C6743AF8
:10805000120050E50D1281C6743A120050E50C1260
:1080600081C6850CF01200B0700FE50CB5F0D5801C
:10807000F4B44103D0A82280F1B42AF51280E812AA
:1080800000B074401281BA90811E1281AFE50E12C9
:108090008155B4180040051280F280E6F50B12807D
:1080A000E874401281BA90812A1281AFE50D1281E5
:1080B00055B43C0040051280F280E6F50A1280E8D3
:1080C00074401281BA9081381281AFE50C1281554B
:1080D000B43C0040051280F280E6750F14F50C8563
:1080E0000A0D850B0E0280301281C090811412811E
:1080F000AF2274001281BA9081461281AF2243757B
:108100007272656E742074696D652069733A00201F
:108110002020200053657420636C6F636B00456EF4
:1081200074657220686F75723A00456E74657220CE
:108130006D696E7574653A00456E7465722073657D
:10814000636F6E643A00496E76616C696420766193
:108150006C756521001281FCF5F07900744E128176
:10816000BAE5F01281E0744EB90101041281BA122D
:1081700000B0700780F91200B380E1B42A09E5F07D
:108180001282081200B322B42A0280EAB43A0050E4
:10819000E5C39430B90001C4C5F0B90004540F80A0
:1081A0000254F045F0F5F009B902CB790080C7E43C
:1081B000936006120050A380F622248012005322FE
:1081C000740102005322C0E0C0F075F00A8443F04D
:1081D000304430120050E5F0120050D0F0D0E022D0
:1081E000C0E0C0F0F5F054F0C42430120050E5F0C7
:1081F000540F2430120050D0F0D0E022C0F075F0BF
:108200000A84C425F0D0F022C0F0C0E054F0C47558
:10821000F00AA4F5F0D0E0540F25F0D0F022C0D041
:10822000C0E0C28C758C4C758A0DD28CD50F21752F
:108230000F14050CE50CB43C17750C00050DE50D8D
:10824000B43C0D750D00050EE50EB41803750E0057
:10825000D0E0D0D032FFFFFFFFFFFFFFFFFFFFFFA7
:00000001FF
